:100000000C94A3040C94BE040C942C1D0C94BE04FC
:100010000C94CE0B0C94DA0A0C94A10B0C94470BA5
:100020000C94740B0C94AD0A0C941A0B0C945A0A91
:100030000C94BE040C9444060C94BE040C940D065F
:100040000C944B0C0C94BE040C94BE040C94BE0493
:100050000C94BE04303132333435363738394142AE
:100060004344454600000001000800400000010034
:100070000400000100080020004000800000010092
:10008000041B63001B5B324A001B5B25646D001B75
:100090005B3F323568001B5B3F32356C001B5B25D4
:1000A000643B25644800636D643E00636D646C6965
:1000B0006E653A2000636F6D6D616E64206E6F74C3
:1000C00020666F756E64007FFF00F700E900DC00BA
:1000D000D000C400B900AF00A5009C0093008B00C5
:1000E00083007C0075006E00680062005D005700B0
:1000F00052004E004900450041003E003A003700E2
:10010000340031002E002C00290027002500230098
:1001100021001F001D001C001A0019001700160006
:10012000150013001200110010000F000F000E0048
:100130000D000C000C000B000A000A00090008006A
:1001400007000600050003000F001F000700030062
:1001500033004F001B007700670037002700630063
:10016000C70047002F0017001300DB0043002300E7
:100170000B005B0133004B009D009B006B005700A0
:1001800001009700B3004D00A700CB0093008B0047
:100190002B000900110099005D00530049002D005B
:1001A00005012D00A3002500210015004500AB002E
:1001B000AD014B0055012B0089009501250153002D
:1001C000A5015501550155102030405060708090B8
:1001D000A0B0C0D0E0F0C4C397757977B58757A5B4
:1001E000A67888D34CE2C2968493B46AA466695A0E
:1001F000865B5976B385A23C6848946774A3F1582E
:100200003955734A4B653D47495483642CC1B24507
:100210002E72922A6337B1463B823A53442D1F38DF
:100220003643523527341C1E621B25A129282B7109
:10023000811D2661171933181A42162432152341DD
:100240001422133112211180858B91989EA5ADB592
:10025000BDC5CEE7E0EAF50D0A57656C636F6D65C5
:1002600020746F2074686520312D426974204772B4
:100270006F6F7665426F78210D0A000D0A3120629A
:1002800069742073796E746820636F6D6D616E643C
:100290007A210D0A004578697465642070726F6771
:1002A00072616D210D0A00417661696C61626C6555
:1002B00020636F6D6D616E6473206172653A0D0A23
:1002C0000068656C702020202020202D2064697338
:1002D000706C61797320617661696C61626C652014
:1002E000636F6D6D616E64730D0A0064756D70618E
:1002F00072677331202D2064756D707320636F6D8C
:100300006D616E6420617267756D656E74732061D6
:100310007320737472696E67730D0A0064756D7073
:100320006172677332202D2064756D707320636F66
:100330006D6D616E6420617267756D656E7473209A
:10034000617320646563696D616C20696E746567B3
:100350006572730D0A0064756D7061726773332086
:100360002D2064756D707320636F6D6D616E6420F8
:10037000617267756D656E7473206173206865784E
:1003800020696E7465676572730D0A007062203CA7
:10039000706F72746220646174613E2D207772699F
:1003A000746520746F20706F727420420D0A0070A3
:1003B00063203C706F72746320646174613E2D2011
:1003C000777269746520746F20706F727420430DAA
:1003D0000A007064203C706F727464206461746100
:1003E0003E2D20777269746520746F20706F72746F
:1003F00020440D0A00756F203C68696768206279A7
:1004000074653E203C6C6F7762797465202D20778F
:1004100072697465206F7574206D61783331303086
:100420002075617274206F6E20706F727420420D9F
:100430000A00616463202D20726561642041444399
:10044000730D0A007369202D2073657175656E63E5
:1004500065722073746172740D0A007373202D200D
:1004600073657175656E6365722073746F700D0AC4
:100470000067202D2067726964736574203C783EA4
:10048000203C793E203C76616C7565200D0A006445
:1004900067202D20646973706C61792067726964CC
:1004A0000D0A0044756D7020617267756D656E741C
:1004B0007320617320737472696E67730D0A004153
:1004C0007267303A2000417267313A20004172670A
:1004D000323A2000417267333A200044756D702033
:1004E000617267756D656E747320617320696E74D7
:1004F00065676572730D0A00417267312061732070
:10050000696E743A20004172673220617320696E0F
:10051000743A20004172673320617320696E743A27
:10052000200044756D7020617267756D656E74731F
:100530002061732068657820696E746567657273E1
:100540000D0A0041726731206173206865783A2096
:100550000041726732206173206865783A2000415B
:10056000726733206173206865783A200025642023
:1005700020202564200025642020202564200D0AE9
:1005800000696E702076616C203D2025640D0A00A4
:10059000696E702076616C203D2025640D0A00256F
:1005A000640D0A0025640D0A0028256429202564AD
:1005B00020202020000D0A00646976506861736570
:1005C0002C2070686173652C206F73634269742CF2
:1005D0002063757257617665666F726D0D0A00252E
:1005E000642C2025642C2025642C2025640D0A0011
:1005F000676C697463684465746563743D25640D54
:100600000A0020000D0A0025642C202D25642D0DE4
:100610000A006E756D436C69636B733D2025640D34
:100620000A00737465707354696C6C4E435A203DB4
:100630002025640D0A000D0A00636F756E746572E3
:10064000477261622020203A2025640D0A007379E8
:100650006E635469636B73477261623A2025640D5F
:100660000A00636C6F636B416363202020202020AD
:100670003A2025642025640D0A007469636B54696F
:100680006D652020202020203A2025642025640D3F
:100690000A006269674F6E652020202020202020FC
:1006A0003A2025640D0A006D617465202020202009
:1006B00020202020203A2025640D0A007474312067
:1006C00020202020202020202020203A20256420C7
:1006D00025640D0A00747432202020202020202060
:1006E000202020203A2025642025640D0A007474FF
:1006F000332020202020202020202020203A2025C8
:10070000642025640D0A00747438202020202020E5
:100710002020202020203A20000D0A007474392067
:1007200020202020202020202020203A20000D0AF8
:10073000007463637230203A2025640D0A007463EC
:10074000637232203A2025640D0A006F63723220F2
:10075000203A2025640D0A00746E6374302072659F
:10076000616C2D74696D65203A2025640D0A007452
:100770006E637431207265616C2D74696D65203A09
:100780002025640D0A00746E637432207265616CFA
:100790002D74696D65203A2025640D0A00636F6D24
:1007A0006253726320282564292C20636F6D62498F
:1007B0006478282564292C20636F6D624465707409
:1007C00068282564290D0A00636F6D624869737497
:1007D000427974654E756D20282564292C20636F3D
:1007E0006D62486973744269744E756D2825642979
:1007F0002C20636F6D624869737442797465282593
:1008000064290D0A00636F6D6248697374426974EC
:1008100020282564290D0A2C00256420000D0A00DB
:100820000D0A206566666563744D6F64653D2564D9
:100830002E2020656666656374566172793D307856
:1008400025780D0A000D0A20636F6D62446570748F
:10085000683D25642E202072706572696F643D25A5
:10086000642E202072696E6770756C736577696499
:100870003D25642E0D0A002564202564006C2A683D
:100880002F64203D2025642025640D0A002D2D2D88
:100890002D2D2D2D2D2D2D2D2D2D2D2D2D2D2D2D88
:1008A0002D0D0A0074656D706F4572726F723A207B
:1008B0002020202020202020000D0A007469636B76
:1008C00054696D653A2020202020202020202020FF
:1008D000000D0A00747269616C4D6174653A2020E4
:1008E0002020202020202020000D0A007469636B46
:1008F00054696D652F747269616C4D6174653A203D
:10090000000D0A006E65774572726F723A202020E2
:100910002020202020202020000D0A006D61674E3D
:1009200065774572726F723A2020202020202020A7
:10093000000D0A00696D70726F76656D656E7421C9
:100940000A000D0A000011241FBECFE5D8E0DEBF6B
:10095000CDBF10E0A0E6B0E0EAE9F4E402C0059003
:100960000D92A83FB107D9F716E0A8EFB0E001C09B
:100970001D92A838B107E1F70C948E0F0C9400007B
:10098000FC01608371834283538316821782148231
:1009900015820895CF93DF93EC01E0E02C813D8137
:1009A00021153105B9F0E881F9818E819F81E80F29
:1009B000F91FE08101968E839F836A817B81861770
:1009C000970720F00E94D3218E839F8321503040CF
:1009D0002C833D838E2F9927DF91CF910895CF935C
:1009E000DF93FC019B01C481D5816C177D07A0F4C6
:1009F00086819781860F971F868397836281738193
:100A00008617970720F00E94D32186839783C21B05
:100A1000D30BC483D58302C014821582DF91CF919A
:100A20000895FC0186819781860F971F228133816B
:100A3000B9010E94D3210190F081E02DE80FF91F48
:100A4000808199270895CF93DF93EC01462F2C8165
:100A50003D816A817B812617370798F48E819F81BB
:100A6000820F931F0E94D321E881F981E80FF91FBB
:100A700040838C819D8101968C839D838FEF90E0D4
:100A800002C080E090E0DF91CF910895FC0140E04A
:100A900050E024813581828193812817390708F439
:100AA00041E0CA010895FC011482158208950E9454
:100AB0007005109279011092780188ED8AB960E88A
:100AC00075E280E090E00E9486058FEF80934704F6
:100AD0001092500410925A04109259047894089578
:100AE00040E450E068EF70E088E494E00E94C004C5
:100AF00040E450E068E371E081E594E00E94C004C6
:100B0000089590937901809378010895DC01CB01D9
:100B100073E0880F991FAA1FBB1F7A95D1F79C011C
:100B2000AD01220F331F441F551F80509C4DAB4019
:100B3000BF4FBC01CD010E94E721DA01C901019735
:100B400089B9892F992780BD089588E494E0089594
:100B500081E594E00895982F809147048823E1F37C
:100B60009CB9109247040895CF93DF93CDB7DEB7B9
:100B700021970FB6F894DEBF0FBECDBFCE01019610
:100B80000E94D205882319F08981992702C08FEF2E
:100B90009FEF21960FB6F894DEBF0FBECDBFDF9159
:100BA000CF910895CF93DF93EC0180914A04909107
:100BB0004B04009769F080914C0490914D0400978C
:100BC00039F088E494E00E94CA0488838FEF90E0B3
:100BD000DF91CF91089510924D0410924C04089526
:100BE00080914C0490914D04892B19F48FEF90E083
:100BF000089580E090E008950895682F81E594E0DD
:100C00000E94230508958FEF8093500481E594E0BE
:100C10000E94CA040E94AB0508951F920F920FB65E
:100C20000F9211242F933F934F935F936F937F9372
:100C30008F939F93AF93BF93EF93FF938091500453
:100C4000882371F08091550490915604892B31F0DE
:100C500081E594E00E94CA048CB905C0109250044A
:100C60008FEF80934704FF91EF91BF91AF919F91D8
:100C70008F917F916F915F914F913F912F910F9045
:100C80000FBE0F901F9018951F920F920FB60F92E4
:100C900011242F933F934F935F936F937F938F9381
:100CA0009F93AF93BF93EF93FF936CB180917801C3
:100CB00090917901892B39F0E0917801F0917901D7
:100CC000862F09950FC088E494E00E9423058823AD
:100CD00049F48091590490915A04019690935A04D2
:100CE00080935904FF91EF91BF91AF919F918F91A4
:100CF0007F916F915F914F913F912F910F900FBE18
:100D00000F901F90189590937B0180937A0108951E
:100D1000CF93DF93EC01892B61F08881882349F020
:100D20008991E0917A01F0917B010995888188236E
:100D3000B9F7DF91CF910895EF92FF920F931F9330
:100D4000CF93DF93EC017A0120E030E0892B01F1B1
:100D5000C9012F5F3F4F8617970718F489918823A1
:100D6000B9F720E030E02E153F0590F48881890125
:100D70000F5F1F4FE0917A01F0917B01882311F002
:100D8000219601C080E2099598010E151F0570F3A8
:100D9000DF91CF911F910F91FF90EF900895CF9326
:100DA000DF93EC01009779F0FC0121968491882370
:100DB00051F0E0917A01F0917B010995FE012196B5
:100DC00084918823B1F7DF91CF910895E0917A0162
:100DD000F0917B018DE00995E0917A01F0917B0122
:100DE0008AE009950895E82FFF27EF70F070EC5A1C
:100DF000FF4F8491E0917A01F0917B01099508956C
:100E00001F93182F82958F700E94F306812F0E94E6
:100E1000F3061F9108950F931F938C01812F99273B
:100E20000E940007802F0E9400071F910F910895D4
:100E3000EF92FF920F931F937B018C01C801AA27A9
:100E4000BB270E940B07C7010E940B071F910F9140
:100E5000FF90EF9008952F923F924F925F926F9282
:100E60007F928F929F92AF92BF92CF92DF92EF923A
:100E7000FF920F931F93CF93DF93CDB7DEB7A29767
:100E80000FB6F894DEBF0FBECDBF69A3C42E2AA350
:100E900027013801442351F017FF08C0EE24FF2436
:100EA0008701E418F5080609170902C083017201D9
:100EB00099A1692F772767FD709561507040CC200C
:100EC00011F061507040D62E18A22FE1222E312C45
:100ED0002C0E3D1E882E992487FC9094A92CB92CA9
:100EE000C801B701A50194010E94E721DC01CB01F3
:100EF000FC01EC5AFF4F84918F8FC801B701A50107
:100F000094010E94E72179018A01DA94EFEFDE165D
:100F100039F1DA94C1010197E114F10401051105D9
:100F2000C1F01C01C801B701A50194010E94E7218D
:100F3000DC01CB01FC01EC5AFF4F8491F10180836D
:100F4000C801B701A50194010E94E72179018A0136
:100F500004C01C018AA1F10180839FEFD916C9F654
:100F6000CC20A9F077FE05C08DE2F10182931F012C
:100F70000EC0C101019714141504160417041CF4C3
:100F80001C018BE202C01C0180E2F1018083D9A028
:100F9000DA94FFEFDF1661F0F10181911F01E0911A
:100FA0007A01F0917B010995DA94FFEFDF16A1F742
:100FB000A2960FB6F894DEBF0FBECDBFDF91CF91E2
:100FC0001F910F91FF90EF90DF90CF90BF90AF9067
:100FD0009F908F907F906F905F904F903F902F9059
:100FE00008957F928F929F92AF92BF92CF92DF929D
:100FF000EF92FF920F931F93CF93DF93CDB7DEB79E
:101000007888C988DA8863E1A62EB12CAC0EBD1EA3
:1010100008C0882309F484C0E0917A01F0917B0133
:10102000099596012F5F3F4F772021F0F601690166
:10103000849103C0F60180816901853251F72F5FE9
:101040003F4F772021F0F6016901849103C0F6013A
:1010500080816901282F332727FD309524363105FB
:1010600091F02536310524F42336310529F0D4CF0B
:101070002837310581F0D0CFF50122E030E0A20E13
:10108000B31E8081C9CF5AE0852E912C40E1E42E19
:1010900047E2F42E04C030E1E32EF12C4701F501C4
:1010A00022E030E0A20EB31E008111818436F1F4FB
:1010B00017FF09C0109501951F4FE0917A01F0913B
:1010C0007B018DE2099532E0E316F10478F00E150C
:1010D0001F0560F4C7016AE070E00E94D3217B0124
:1010E0006230710518F006171707A0F3C801B701A1
:1010F0000E94D321FB01EC5AFF4F8491E0917A01C9
:10110000F0917B010995C801B7010E94D3218C01A0
:10111000C701B4010E94D3217B01672B39F781CF2E
:1011200080E090E0DF91CF911F910F91FF90EF90C1
:10113000DF90CF90BF90AF909F908F907F90089559
:10114000E0917A01F0917B0109950895039665E09D
:1011500070E00E94D321CB01AA27BB2724E0880F8F
:10116000991FAA1FBB1F2A95D1F720E030E028174E
:10117000390728F42F5F3F4F28173907D8F3089510
:10118000CF93C0E08C2F0E943009CF5FC830D0F3DE
:101190000E94D1080E94DB080E94E4087894CF9155
:1011A000089582E00E94EE0812BE89B7816089BF6F
:1011B0000E94D909089583E00E94F4081DBC1CBC5C
:1011C00089B7846089BF089584E00E94FA0814BC3E
:1011D00089B7806489BF0E94ED090895982F83B76D
:1011E000887F892B83BF0895982F8EB5887F892BA0
:1011F0008EBD0895982F85B5887F892B85BD08956C
:1012000083B7E82FFF27E770F070EE0FFF1FEB5951
:10121000FF4F8591949108958EB5E82FFF27E770D1
:10122000F070EE0FFF1FEB59FF4F859194910895D9
:1012300085B5E82FFF27E770F070EE0FFF1FEF581E
:10124000FF4F859194910895883040F4E82FFF274F
:10125000EE0FFF1FE458FE4F6083718308950895D9
:10126000883040F4E82FFF27EE0FFF1FE458FE4FB1
:101270001082118208950895DF92EF92FF920F93EA
:101280001F93CF93DF93EC01D2B610925F041092BC
:10129000600410926104109262040E9400099C0193
:1012A0004427552760E074E284EF90E00E94092211
:1012B000293B8DE8380786E0480780E05807C0F4EE
:1012C00087E2C131D807A0F4CE01AA27BB27BC0111
:1012D000CD010E94B421DC01CB01BC01CD0128EE7F
:1012E00033E040E050E00E94E721FA01E90111C03B
:1012F0007E0100271127CA01B90128EE33E040E042
:1013000050E00E94E721C801B7010E94B421FC010E
:10131000EB0180915F0490916004A0916104B09111
:1013200062042227382F492F5A2F82B79927AA27DC
:10133000BB27282B392B4A2B5B2BCD0DD11DE11D53
:10134000F11D2C173D074E075F0758F580915F048C
:1013500090916004A0916104B091620485B78F7888
:1013600085BF85B7806885BF889585B78F7785BF2E
:1013700080915F0490916004A0916104B091620437
:101380002227382F492F5A2F82B79927AA27BB2700
:10139000282B392B4A2B5B2B2C173D074E075F0759
:1013A000A8F2DF91CF911F910F91FF90EF90DF9006
:1013B000089510925B0410925C0410925D041092E8
:1013C0005E04089580915B0490915C04A0915D049B
:1013D000B0915E04BC01CD01089510926304109297
:1013E0006404109265041092660408958091630469
:1013F00090916404A0916504B0916604BC01CD0194
:101400000895893031F48FB582608FBD8FB58E7F9E
:101410000AC08A3019F48FB5826002C08FB58D7F03
:101420008FBD8FB581608FBD1BBC1ABC19BC18BCA9
:1014300008959C018FB58E7F8FBD8FB582608FBD63
:101440008EB588608EBD8EB580618EBD37BD26BDE0
:101450001BBC1ABC19BC18BC08958FB58D7F8FBDFD
:101460008FB58E7F8FBD0E94460A0E944D0A089557
:101470008FB580688FBD8FB58F7B8FBD08958FB579
:1014800080628FBD8FB58F7E8FBD08958FB58F77AA
:101490008FBD8FB58F7B8FBD08958FB58F7D8FBD2D
:1014A0008FB58F7E8FBD08959BBD8ABD089599BD70
:1014B00088BD08951F920F920FB60F9211242F939B
:1014C0003F934F935F936F937F938F939F93AF93CC
:1014D000BF93EF93FF9380915B0490915C04A09184
:1014E0005D04B0915E040196A11DB11D80935B0463
:1014F00090935C04A0935D04B0935E0480915F04BC
:1015000090916004A0916104B09162040196A11DC4
:10151000B11D80935F0490936004A0936104B09325
:10152000620480917C0190917D01892B29F0E091EA
:101530007C01F0917D010995FF91EF91BF91AF91F1
:101540009F918F917F916F915F914F913F912F91DB
:101550000F900FBE0F901F9018951F920F920FB60D
:101560000F9211242F933F934F935F936F937F9329
:101570008F939F93AF93BF93EF93FF9380917E01DF
:1015800090917F01892B29F0E0917E01F0917F01FC
:101590000995FF91EF91BF91AF919F918F917F91AD
:1015A0006F915F914F913F912F910F900FBE0F90D0
:1015B0001F9018951F920F920FB60F9211242F9320
:1015C0003F934F935F936F937F938F939F93AF93CB
:1015D000BF93EF93FF938091630490916404A09173
:1015E0006504B09166040196A11DB11D809363044A
:1015F00090936404A0936504B0936604809186017F
:1016000090918701892B29F0E0918601F091870163
:101610000995FF91EF91BF91AF919F918F917F912C
:101620006F915F914F913F912F910F900FBE0F904F
:101630001F9018951F920F920FB60F9211242F939F
:101640003F934F935F936F937F938F939F93AF934A
:10165000BF93EF93FF9380918A0190918B01892B27
:1016600029F0E0918A01F0918B010995FF91EF91AA
:10167000BF91AF919F918F917F916F915F914F91AA
:101680003F912F910F900FBE0F901F9018951F92B2
:101690000F920FB60F9211242F933F934F935F93A6
:1016A0006F937F938F939F93AF93BF93EF93FF932A
:1016B0008091800190918101892B29F0E091800136
:1016C000F09181010995FF91EF91BF91AF919F91A9
:1016D0008F917F916F915F914F913F912F910F90DB
:1016E0000FBE0F901F9018951F920F920FB60F927A
:1016F00011242F933F934F935F936F937F938F9317
:101700009F93AF93BF93EF93FF938091820190914A
:101710008301892B29F0E0918201F09183010995E1
:10172000FF91EF91BF91AF919F918F917F916F91B9
:101730005F914F913F912F910F900FBE0F901F908F
:1017400018951F920F920FB60F9211242F933F936B
:101750004F935F936F937F938F939F93AF93BF93B9
:10176000EF93FF938091840190918501892B29F05B
:10177000E0918401F09185010995FF91EF91BF916E
:10178000AF919F918F917F916F915F914F913F9119
:101790002F910F900FBE0F901F9018951F920F92D0
:1017A0000FB60F9211242F933F934F935F936F9334
:1017B0007F938F939F93AF93BF93EF93FF9380910A
:1017C000880190918901892B29F0E0918801F0919D
:1017D00089010995FF91EF91BF91AF919F918F91F1
:1017E0007F916F915F914F913F912F910F900FBE1D
:1017F0000F901F901895379A359886E00E940C0C30
:1018000081E00E94120C3D98339A109267047894FC
:101810000895339837980895982F86B1887F892B3B
:1018200086B9089527B12F73992736E0880F991F3D
:101830003A95E1F7282B27B90895982F87B1807E34
:101840009F71892B87B90895349A369A089586B185
:101850009927807490700895982F1092670487B12B
:10186000807E9F71892B87B9349A369A3699FECF3C
:1018700084B1282F332785B19927982F8827282BC3
:10188000392BC90108950E942C0C96958795969541
:101890008795992708951F920F920FB60F921124E2
:1018A0008F938FEF809367048F910F900FBE0F90EF
:1018B0001F90189581E890E00E94CF06089584E873
:1018C00090E00E94CF06089599279F938F9389E80F
:1018D00090E09F938F9381E08F930E94F1070F9088
:1018E0000F900F900F900F900895882319F08FE8B4
:1018F00090E002C086E990E09F938F9381E08F9300
:101900000E94F1070F900F900F900895282F862FB7
:1019100099279F938F93822F99279F938F938DE978
:1019200090E09F938F9381E08F930E94F1078DB792
:101930009EB707960FB6F8949EBF0FBE8DBF089551
:1019400010926C041092680410926D0410926A0454
:101950001092690410926B0408950F931F939C01D9
:101960008B0190916B048FE0989FC00111248457E4
:101970009E4FB9010E944F2080916B04E82FFF27F2
:10198000EE0FFF1FEC51FC4F008311838F5F80939C
:101990006B041F910F910895909335048093340444
:1019A00008951F93CF93182F20916C04223009F0D3
:1019B00045C099278234910581F08334910524F440
:1019C0008134910541F037C08334910551F084345E
:1019D000910511F130C081E001C0822F0E942A0ED2
:1019E0002AC090916D0480916804E0913404F091D4
:1019F00035049817F0F49F5F90936D048BE109957F
:101A0000E0913404F09135048BE50995E0913404BC
:101A1000F091350483E40EC080916D04E0913404AC
:101A2000F0913504882329F0815080936D0488E07B
:101A300001C087E0099510926C04E9C0213021F4BF
:101A40008B3511F482E0E1C010926C04812F80523A
:101A50008F3508F04BC090916D0480916804981701
:101A6000B1F4E0913404F0913504812F099580910F
:101A70006D04E82FFF27E259FB4F10838F5F80939F
:101A80006D04809168048F5F80936804C0C08F5F8D
:101A900080936804C82F981750F4EC2FFF27E25961
:101AA000FB4F829131968083C1509C17B0F3809197
:101AB0006D04E82FFF27E259FB4F10838F5F80935F
:101AC0006D040E940A0EC0916D0480916804C817CD
:101AD00008F09DC0E0913404F091350488E0099548
:101AE000CF5F80916804C817A8F391C01D3011F52D
:101AF000E0913404F0913504812F0995E09134048C
:101B0000F09135048AE0099580916804E82FFF2759
:101B1000E259FB4F10828F5F8093680480916D04BF
:101B20008F5F80936D040E94540E1092680410928F
:101B30006D046DC0183009F063C080916D04882376
:101B400009F457C0909168048917E9F4E0913404CE
:101B5000F0913504812F0995E0913404F09135041A
:101B600080E20995E0913404F0913504812F0995C4
:101B70008091680481508093680480916D04815045
:101B800080936D0444C09150909368048150809379
:101B90006D04C82F891748F4EC2FFF27E259FB4F3B
:101BA00081818083CF5FC917B8F30E940A0EE0914C
:101BB0003404F091350480E20995C0916D042C2F16
:101BC0003327809168049927019628173907FCF478
:101BD000E0913404F091350488E00995CF5F2C2F13
:101BE000332780916804992701962817390784F3D1
:101BF0000EC0E0913404F091350487E0099507C0E8
:101C00001F3729F01B3119F481E080936C04CF91C8
:101C10001F9108950F931F93CF93E0913404F09197
:101C200035048DE009950E94A80EC09168040EE667
:101C300014E0C150CF3F51F0F80181918F01E09144
:101C40003404F09135040995C150B0F7CF911F913C
:101C50000F91089599278130910581F08230910587
:101C60000CF5892BF9F480916E048823D9F06EE687
:101C700074E08EEB94E00E944F2008956EEB74E0C8
:101C80008EE694E00E944F20EEE6F4E00190002002
:101C9000E9F73197EE56F440E0936804E0936D0461
:101CA0000E940A0E089508951F93CF9310E0812F8C
:101CB0000E942A0E80916E04803261F0882351F0D8
:101CC0001F5FE12FFF27E259FB4FE081E03211F067
:101CD000EE23B1F7112371F427C0EC2FFF27EE0F8D
:101CE000FF1FEC51FC4F8081918190936A04809397
:101CF00069041CC0C0E080916B04C81798F48FE0A1
:101D0000C89FC001112484579E4F412F55276EE66E
:101D100074E00E945620892B01F3CF5F80916B0401
:101D2000C81768F30E94BF0E0E94A80ECF911F91A2
:101D30000895E0916904F0916A04309739F00995AB
:101D400010926A04109269040E94A80E08950895E2
:101D5000CF93DF93C6EAD0E0FE018491882361F03F
:101D6000FE0121968491E0913404F09135040995A7
:101D7000FE0184918823A1F7DF91CF910895CF933D
:101D8000DF93CBEAD0E0FE018491882361F0FE016D
:101D900021968491E0913404F09135040995FE0177
:101DA00084918823A1F7CEE6D4E080916E04882345
:101DB00069F0803259F08991E0913404F091350452
:101DC00009958881882311F08032A9F7E0913404C5
:101DD000F09135048AE30995E0913404F0913504DB
:101DE00080E20995C5EBD0E0FE018491882361F083
:101DF000FE0121968491E0913404F0913504099517
:101E0000FE0184918823A1F7E0913404F091350418
:101E10008DE00995E0913404F09135048AE009954C
:101E2000DF91CF910895382F90E080916E04803239
:101E300041F49F5FE92FFF27E259FB4F80818032F9
:101E4000C1F320E0231728F5E92FFF27E259FB4FC4
:101E5000E081EE2361F0E03251F09F5FE92FFF2730
:101E6000E259FB4FE081EE2311F0E032B1F7E92FA8
:101E7000FF27E259FB4F8081803241F49F5FE92FB9
:101E8000FF27E259FB4F80818032C1F32F5F231778
:101E9000D8F2892F992782599B4F0895CF93DF93CA
:101EA000CDB7DEB722970FB6F894DEBF0FBECDBF19
:101EB0000E94130F4AE050E0BE016F5F7F4F0E9407
:101EC0006420DC01CB01BC01CD0122960FB6F89451
:101ED000DEBF0FBECDBFDF91CF910895CF93DF93CB
:101EE000CDB7DEB722970FB6F894DEBF0FBECDBFD9
:101EF0000E94130F40E150E0BE016F5F7F4F0E94D0
:101F00006420DC01CB01BC01CD0122960FB6F89410
:101F1000DEBF0FBECDBFDF91CF910895CFE5D8E0F2
:101F2000DEBFCDBF0E94570560E071EE80E090E01B
:101F30000E9486058BEA95E00E9483060E94FB0BB7
:101F40000E94C0080E945A0C87E592E09F938F93ED
:101F500081E08F930E94F1071ABA87EF8BBB8FE065
:101F600087BB80EF88BB14BA8FEF85BB11BA82BBE9
:101F70000E9423170F900F900F90E6E3F5E09F016A
:101F800028503F4F80E4808338962E173F07D4F7C0
:101F90000E94A61A0E94D00F80E090E00C944C2280
:101FA000CF93DF93CDB7DEB721970FB6F894DEBF9E
:101FB0000FBECDBF0E945F0C60E081E00E94860CE6
:101FC0008BE792E00E94CF060E94A00C8BEA95E07E
:101FD0000E94CC0C6BEB70E18EE790E00E94AD0CA0
:101FE0006FE471E183E890E00E94AD0C6DE871E16F
:101FF0008DE890E00E94AD0C63EF71E187E990E01D
:102000000E94AD0C69E572E181EA90E00E94AD0C9E
:102010006DE572E186EA90E00E94AD0C6AE972E13A
:102020008BEA90E00E94AD0C6CEA72E18EEA90E0DF
:102030000E94AD0C66EC72E181EB90E00E94AD0C69
:1020400060EE72E184EB90E00E94AD0C64EF72E10F
:1020500087EB90E00E94AD0C61E672E18BEB90E0C3
:102060000E94AD0C6DEC73E18EEB90E00E94AD0C24
:1020700068E174E181EC90E00E94AD0C6FEE7AE1D2
:1020800083EC90E00E94AD0C66EA7AE186EC90E089
:102090000E94AD0C6AE374E189EC90E00E94AD0C03
:1020A00063E97EE18FEC90E00E94AD0C6CE673E199
:1020B00083ED90E00E94AD0C65E873E187ED90E060
:1020C0000E94AD0C6DE873E18BED90E00E94AD0CC9
:1020D0006CEA73E18FED90E00E94AD0C66EB73E16A
:1020E00084EE90E00E94AD0C6EEB73E188EE90E020
:1020F0000E94AD0C66E273E18BEE90E00E94AD0CA5
:1021000069E370E28EEE90E00E94AD0C62EE76E143
:1021100081EF90E00E94AD0C8DE00E94D10C8FEF1A
:102120008093100503C089810E94D10CCE010196D5
:102130000E94D2058823B9F70E94990E809110055C
:102140008823A1F70E94E60685E992E09F938F938A
:1021500081E08F930E94F1070F900F900F902196CE
:102160000FB6F894DEBF0FBECDBFDF91CF910895BB
:102170001092100508951F930E94E60687EA92E0E8
:102180009F938F9311E01F930E94F1070F900F9080
:102190000F9081EC92E09F938F931F930E94F10721
:1021A0000F900F900F908BEE92E09F938F931F9361
:1021B0000E94F1070F900F900F908CE193E09F9396
:1021C0008F931F930E94F1070F900F900F9086E559
:1021D00093E09F938F931F930E94F1070F900F90AE
:1021E0000F908CE893E09F938F931F930E94F107C9
:1021F0000F900F900F908FEA93E09F938F931F9310
:102200000E94F1070F900F900F9082ED93E09F9343
:102210008F931F930E94F1070F900F900F9085EFFF
:1022200093E09F938F931F930E94F1070F900F905D
:102230000F9082E394E09F938F931F930E94F10786
:102240000F900F900F9084E494E09F938F931F93CF
:102250000E94F1070F900F900F908BE594E09F93F1
:102260008F931F930E94F1070F900F900F9081E7BB
:1022700094E09F938F931F930E94F1070F900F900C
:102280000F908FE894E09F938F931F930E94F10724
:102290000E94E6060F900F900F901F9108951F93D4
:1022A0000E94E60683EA94E09F938F9311E01F93C8
:1022B0000E94F1070F900F900F908FEB94E00E9417
:1022C000CF0680E00E94130F0E9488060E94E60657
:1022D00086EC94E00E94CF06812F0E94130F0E948B
:1022E00088060E94E6068DEC94E00E94CF0682E00C
:1022F0000E94130F0E9488060E94E60684ED94E077
:102300000E94CF0683E00E94130F0E9488060E945D
:10231000E6060E94E6061F910895DF92EF92FF9273
:102320000F931F930E94E6068BED94E09F938F938B
:1023300081E0D82EDF920E94F1070F900F900F904E
:1023400088EF94E09F938F93DF920E94F1078D2D89
:102350000E944E0FDC01CB017C018D0120E24FEF8A
:102360006AE0862F0E942B070E94E6060F900F90CE
:102370000F9086E095E09F938F93DF920E94F10784
:1023800082E00E944E0FDC01CB017C018D0120E236
:102390004FEF6AE0862F0E942B070E94E6060F90FF
:1023A0000F900F9084E195E09F938F93DF920E94AE
:1023B000F10783E00E944E0FDC01CB017C018D010F
:1023C00020E24FEF6AE0862F0E942B070E94E6066C
:1023D0000E94E6060F900F900F901F910F91FF90B3
:1023E000EF90DF900895DF92EF92FF920F931F938B
:1023F0000E94E60682E295E09F938F9391E0D92EAA
:10240000DF920E94F1070F900F900F9083E495E008
:102410009F938F93DF920E94F1078D2D0E946E0F84
:10242000DC01CB017C018D0120E240E068E080E12D
:102430000E942B070E94E6060F900F900F9081E5F7
:1024400095E09F938F93DF920E94F10782E00E94B4
:102450006E0FDC01CB017C018D0120E240E068E0E1
:1024600080E10E942B070E94E6060F900F900F90CC
:102470008FE595E09F938F93DF920E94F10783E0B1
:102480000E946E0FDC01CB017C018D0120E240E057
:1024900068E080E10E942B070E94E6060E94E606A3
:1024A0000F900F900F901F910F91FF90EF90DF9082
:1024B000089580E00E94120C089581E00E94120CA1
:1024C0000895FF920F931F9329B386B3F3B200B31D
:1024D00099279F938F93822F99279F938F938DE6B0
:1024E00095E09F938F9311E01F930E94F1078DB7A2
:1024F0009EB707960FB6F8949EBF0FBE8DBF802F74
:1025000099279F938F938F2D99279F938F9386E77A
:1025100095E09F938F931F930E94F1078DB79EB70D
:1025200007960FB6F8949EBF0FBE8DBF1F910F91F7
:10253000FF90089589B399279F938F9381E895E041
:102540009F938F9381E08F930E94F1070F900F90DC
:102550000F900F900F9008951F9386B399279F9324
:102560008F9380E995E09F938F9311E01F930E94D2
:10257000F107812F0E944E0FDC01CB0188BB0F9029
:102580000F900F900F900F901F9108951F9383B39A
:1025900099279F938F938FE995E09F938F9311E0F5
:1025A0001F930E94F107812F0E944E0FDC01CB0187
:1025B00085BB0F900F900F900F900F901F91089573
:1025C0000E94E60680B399279F938F9384EA95E053
:1025D0009F938F9381E08F930E94F1070F900F904C
:1025E0000F900F900F9008950F931F93CF93DF9349
:1025F00010E0C1E0D0E0812F0E94430C99279F9307
:102600008F93DF93CF9389EA95E09F938F9301E0B7
:102610000F930E94F1078DB79EB707960FB6F894F7
:102620009EBF0FBE8DBF100F2196183020F385EB93
:1026300095E09F938F930F930E94F1070F900F9057
:102640000F90DF91CF911F910F9108951F9388EB09
:1026500095E09F938F9311E01F930E94F1070F90D5
:102660000F900F9080916E0690916F069F938F93BD
:102670008091560699279F938F93809142069927C0
:102680009F938F9380913406909135069F938F93FB
:102690008FED95E09F938F931F930E94F1078DB765
:1026A0009EB70B960FB6F8949EBF0FBE8DBF80915C
:1026B000400499279F938F9380EF95E09F938F938A
:1026C0001F930E94F107109240040F900F900F90FB
:1026D0000F900F901F91089581E00E944E0FDC0132
:1026E000CB01880F991FFC01E95BFE4F2491332732
:1026F000322F2227885B9E4FFC018491280F311DC9
:1027000030936F0620936E06089581E00E944E0F6D
:10271000DC01CB0180936106089581E00E944E0F99
:10272000DC01CB01992790935506809354069C01B8
:10273000280F391FF901E953FF4F84919927982FEA
:10274000882728533F4FF9012491820F911D9093C0
:10275000590680935806089581E00E944E0FDC01CF
:10276000CB0190930F0580930E05089581E00E94A0
:102770004E0FDC01CB0180935106089581E00E9449
:102780004E0FDC01CB01982F9F73909336048295F6
:1027900086958770809360000895AF92BF92CF9224
:1027A000DF92EF92FF920F931F93CF93DF93AA24B0
:1027B000BB24E501CD5CDA4F6FE1C62ED12C8881B8
:1027C00028969927AA27BB277C018D0120E340E0AA
:1027D00062E080E10E942B0782E096E09F938F9356
:1027E00011E01F930E94F1070F900F900F90089433
:1027F000C108D108D7FEE3CF84E096E09F938F9382
:102800001F930E94F1070F900F900F900894A11C46
:10281000B11C84E0A816B10464F2DF91CF911F913E
:102820000F91FF90EF90DF90CF90BF90AF90089501
:102830000F931F9381E00E944E0FDC01CB01082F04
:1028400082E00E944E0FDC01CB01182F83E00E9432
:102850004E0FDC01CB01E02FFF2773E0EE0FFF1FCF
:102860007A95E1F7ED5CFA4FE10FF11D80831F913E
:102870000F9108950F931F93CF93DF9380913D069F
:1028800099279F938F9380913F0499279F938F93CC
:1028900087E096E09F938F9311E01F930E94F107CA
:1028A0004DB75EB7495F5F4F0FB6F8945EBF0FBE7E
:1028B0004DBF8091700699279F938F9382E196E098
:1028C0009F938F931F930E94F1070F900F900F908B
:1028D0000F900F9080917C0090917D009F938F933B
:1028E00082E296E09F938F931F930E94F1070F90CF
:1028F0000F900F900F900F9086E396E09F938F9329
:102900001F930E94F1070F900F900F908091520635
:1029100099279F938F9389E396E09F938F931F93BB
:102920000E94F1070F900F900F900F900F908091E1
:102930005F06909160069F938F938EE496E09F933D
:102940008F931F930E94F10780913E0690913F065E
:10295000A0914006B0914106CD01AA27BB27209146
:102960003E0630913F060F900F900F900F900F9002
:102970003F932F939F938F9382E696E09F938F933D
:102980001F930E94F1078091180590911905A0915D
:102990001A05B0911B05CD01AA27BB272091180568
:1029A000309119054DB75EB7495F5F4F0FB6F89488
:1029B0005EBF0FBE4DBF3F932F939F938F938AE7C8
:1029C00096E09F938F931F930E94F1078DB79EB758
:1029D00007960FB6F8949EBF0FBE8DBF8091720010
:1029E000909173009F938F9382E996E09F938F93CA
:1029F0001F930E94F1070F900F900F900F900F9070
:102A000080917400909175009F938F9387EA96E070
:102A10009F938F931F930E94F10780915A06909184
:102A20005B06A0915C06B0915D06CD01AA27BB278D
:102A300020915A0630915B060F900F900F900F90E7
:102A40000F903F932F939F938F938CEB96E09F93E0
:102A50008F931F930E94F1078091110590911205A9
:102A6000A0911305B0911405CD01AA27BB27209191
:102A70001105309112054DB75EB7495F5F4F0FB634
:102A8000F8945EBF0FBE4DBF3F932F939F938F93DC
:102A900085ED96E09F938F931F930E94F10780919D
:102AA0002C0590912D05A0912E05B0912F05CD01FB
:102AB000AA27BB2720912C0530912D054DB75EB775
:102AC000495F5F4F0FB6F8945EBF0FBE4DBF3F9397
:102AD0002F939F938F938EEE96E09F938F931F93E8
:102AE0000E94F1078DB79EB707960FB6F8949EBF68
:102AF0000FBE8DBF87E097E09F938F931F930E9437
:102B0000F1078091820690918306A0918406B0918E
:102B10008506BC01CD010E94C8160F900F900F9042
:102B200089E197E09F938F931F930E94F1070F9085
:102B30000F900F908CE197E09F938F931F930E94CB
:102B4000F1078091480690914906A0914A06B091FC
:102B50004B06BC01CD010E94C8160F900F900F903C
:102B60008EE297E09F938F931F930E94F1070F903F
:102B70000F900F9083B799279F938F9381E397E0EE
:102B80009F938F931F930E94F1070F900F900F90C8
:102B90000F900F9085B599279F938F938EE397E0C1
:102BA0009F938F931F930E94F1070F900F900F90A8
:102BB0000F900F9083B599279F938F938BE497E0A5
:102BC0009F938F931F930E94F1070F900F900F9088
:102BD0000F900F9082B799279F938F9388E597E086
:102BE0009F938F931F930E94F1070F900F900F9068
:102BF0000F900F908CB59DB59F938F938FE697E0C4
:102C00009F938F931F930E94F1070F900F900F9047
:102C10000F900F9084B599279F938F9386E897E044
:102C20009F938F931F930E94F1070F900F900F9027
:102C30000F900F9080916B0699279F938F938091AF
:102C4000750699279F938F938091330699279F93B9
:102C50008F938DE997E09F938F931F930E94F107C5
:102C60004DB75EB7475F5F4F0FB6F8945EBF0FBEBC
:102C70004DBF8091570699279F938F93809115059B
:102C800099279F938F938091470699279F938F93BE
:102C900088EC97E09F938F931F930E94F1078DB765
:102CA0009EB709960FB6F8949EBF0FBE8DBF809158
:102CB000620699279F938F9385E098E09F938F9367
:102CC0001F930E94F10710E00F900F900F900F904C
:102CD0000F90CAE7D6E0899199279F938F9389E156
:102CE00098E09F938F9301E00F930E94F1070F905C
:102CF0000F900F900F900F90100F183060F38DE130
:102D000098E09F938F930F930E94F1070F900F907D
:102D10000F908091360499279F938F938091600044
:102D200099279F938F9380E298E09F938F930F93BF
:102D30000E94F1074DB75EB7495F5F4F0FB6F89439
:102D40005EBF0FBE4DBF80913105909132059F93BC
:102D50008F9380910E0590910F059F938F93809193
:102D60006B0699279F938F9385E498E09F938F93A9
:102D70000F930E94F1078DB79EB709960FB6F8948E
:102D80009EBF0FBE8DBFDF91CF911F910F91089510
:102D9000DC01CB019D01442755279F938F933F93DF
:102DA0002F9387E798E09F938F9381E08F930E9402
:102DB000F1078DB79EB707960FB6F8949EBF0FBE6A
:102DC0008DBF0895AF92BF92CF92DF92EF92FF92A4
:102DD0000F931F9381E00E944E0F7B018C0182E0D4
:102DE0000E944E0FDC01CB01E81AF90A0A0B1B0BFB
:102DF0005801CC24DD24C801B7010E94C816D801AF
:102E0000C701BF77BC01CD010E94C816FF92EF92A7
:102E1000BF92AF928DE798E09F938F9381E08F935D
:102E20000E94F1078DB79EB707960FB6F8949EBF24
:102E30000FBE8DBF1F910F91FF90EF90DF90CF904D
:102E4000BF90AF90089581E090E0909359068093F1
:102E50005806109235061092340610926F061092A2
:102E60006E068BE0809361061092420610920F0569
:102E700010920E05109217051092160580E090E84A
:102E8000909332058093310581E080935106089537
:102E9000CF930E941B2080913406909135060196B5
:102EA0009093350680933406209158063091590648
:102EB0008217930700F11092350610923406809124
:102EC00042068F5F8093420690916106891710F049
:102ED0001092420680916E0690916F060090420615
:102EE00002C0969587950A94E2F78170907090934E
:102EF00042048093410440914104409356066091FE
:102F00006000862F992783309105D1F08430910598
:102F10003CF481309105A1F002970CF06DC069C1BD
:102F20008530910509F4B2C0853091050CF47FC05D
:102F30008630910509F4D7C0079709F40CC159C12F
:102F40004091750680916B06242F281B822F8F736A
:102F50008695869586952770E82FFF27E658F94FC6
:102F60008081992702C0959587952A95E2F781700F
:102F700080936206C09156065C2F582750935606E0
:102F800040933306842F86958695869580934706D1
:102F9000942F977090931505E82FFF27E658F94F67
:102FA000E081292F332781E090E0022E02C0880FB4
:102FB000991F0A94E2F78095E823E0935706613061
:102FC00019F48C2F992702C0852F992702C0880FEA
:102FD000991F2A95E2F7E82BE09357068091470660
:102FE000E82FFF27E658F94F8091570680834F5FFF
:102FF0004F7340937506FDC080911605909117059B
:1030000020910E0530910F05820F931F90931705A5
:103010008093160520913105309132052817390724
:1030200008F0E7C081E0482740935606E2C080914F
:10303000390490913A04019690933A0480933904AC
:1030400020916700309168008217930708F4D1C07F
:1030500010923A041092390480913B048F5F809360
:103060003B0490916900891710F010923B04809105
:103070003B04E82FFF27EE0FFF1FE659FF4F80812B
:1030800091819093590680935806B3C0C42F209124
:103090006C0030916D0036952795809116059091C2
:1030A0001705820F931F909317058093160597FDC0
:1030B000CF5F20916E0030916F0036952795369541
:1030C000279580913D0490913E04820F931F909329
:1030D0003E0480933D0497FDCF5F10925606C230A8
:1030E00008F487C083C060913C04862F99274091E3
:1030F0003D0450913E042091700030917100892B65
:1031000079F4CA01820F931F90933E0480933D048B
:103110004DE781309407C8F0821B930B09970DC0CF
:10312000CA01821B930B90933E0480933D044DE7AC
:103130008130940750F0820F931F90933E04809348
:103140003D0481E0861B80933C0480913C048823ED
:1031500009F04FC04CC08091160590911705209141
:103160000E0530910F05820F931F909317058093E2
:103170001605C42F209131053091320528173907E3
:1031800008F4CF5FC295C07F8091370490913804D6
:103190000196909338048093370420916500309114
:1031A00066008217930730F00E94021910923804CB
:1031B0001092370440913606809161009091620030
:1031C0002091630030916400820F931F849F9001CF
:1031D0001124232F33274695842F99274096109248
:1031E00056062C0F311D2817390718F081E08093FF
:1031F000560680915606882311F4C39801C0C39ADD
:10320000CF9108958091610090916200BC01662782
:10321000770F661F77279C012070307424E0329F5F
:10322000212D33271124AC0140705071452F5527B3
:1032300042954F702627372724273527880F991F57
:10324000822B932B90936200809361002091630006
:1032500030916400B9016070707464E0769F612DF4
:1032600077271124C90180709072892F9927829540
:103270008695877068277927220F331F262B372BD7
:10328000309364002093630008959927880F991F55
:10329000FC01E95BFE4F24913327322F2227885B04
:1032A0009E4FFC018491280F311D30936F062093AF
:1032B0006E060895809361060895992790935506A8
:1032C000809354069C01280F391FF901E953FF4FE1
:1032D00084919927982F882728533F4FF9012491EB
:1032E000820F911D909359068093580608958095FA
:1032F000869586958F5F80936B060895482F40953D
:1033000046954695842F9927880F991FFC01E9530C
:10331000FF4F24913327322F222788539F4FFC01E0
:103320008491280F311D53E0220F331F5A95E1F786
:103330004F3311F420E030E030930F0520930E0559
:10334000089599279C01369527959695982F88275B
:1033500097958795822B932B909332058093310517
:1033600008958093510608958695869599278770CC
:1033700090708330910529F1843091054CF48130AF
:103380009105A9F082309105CCF4892B69F008955C
:1033900085309105E1F085309105B4F086309105D6
:1033A000C9F00797D1F0089581E090E002C082E073
:1033B00090E09093660080936500089583E090E02C
:1033C000F8CF84E090E0F5CF87E090E0F2CF83E1A2
:1033D00090E0EFCF8DE390E0ECCF82ED94E0E9CF89
:1033E000809336060895482F809350064695809125
:1033F000540690915506880F991FFC01E953FF4F21
:1034000024913327322F222788539F4FFC01849128
:10341000280F311D30936B0020936A00E42FFF27A3
:10342000E953FE4F5491852F82958F704091540639
:10343000480F403408F04C50403408F04C50842F72
:103440009927880F991FFC01E953FF4F24913327D7
:10345000322F222788539F4FFC018491280F311D62
:1034600030936D0020936C00952F9F7021F482E0C3
:10347000809369001FC083E080936900940F9034AB
:1034800008F09C50903408F09C50892F9927880FA1
:10349000991FFC01E953FF4F24913327322F222734
:1034A00088539F4FFC018491280F311D30936F008A
:1034B00020936E0080913B04E82FFF27EE0FFF1F43
:1034C000E659FF4F80819181909359068093580669
:1034D0000895482F4095E42FFF27EF70F070E95BC7
:1034E000FD4F84919927382F222742954F708FE006
:1034F00090E0841B910902C0369527958A95E2F7E2
:103500002F5F3F4F30936800209367000895482F46
:10351000E82FFF27EF70F070E95BFD4F849199274A
:10352000382F222742954F708FE090E0841B91093D
:1035300002C0369527958A95E2F7369527953695F8
:1035400027953093710020937000089589B78D7F7F
:1035500089BF68E477E187E00E9424098AE083BF9D
:103560008DE28CBF89B7826089BF89B78F7E89BFA2
:1035700069EF7AE182E00E94240920917200309183
:103580007300832F99278BBD2ABD89E08EBD1FBC98
:1035900089B7806189BF89B78F7789BF62E27DE192
:1035A00086E00E9424098CE085BD8091760083BD71
:1035B00089B7806889BF1092700610923E061092FB
:1035C0003F06109240061092410685B7886085BF7D
:1035D00085B78E7F85BF8BB780688BBF089589B70D
:1035E0008D7F89BF89B78F7E89BF89B78F7789BF64
:1035F0000895809145049091460401969093460465
:10360000809345042091F6003091F70082179307CC
:10361000D4F0109246041092450480914304909196
:1036200044040196909344048093430420917400D1
:10363000309175008217930730F010924404109275
:1036400043040E94241B089580913F048F5F8F7173
:1036500080933F040E94401B80917C0090917D00EC
:10366000019790937D0080937C0097FF06C0109295
:103670007D0010927C00109270060E94E81B089555
:10368000CF9380913F04E82FFF2723E0EE0FFF1F29
:103690002A95E1F7ED5CFA4FC0818C2F0E94451905
:1036A000CC0FCC0FC093240580913F04E82FFF2757
:1036B00093E0EE0FFF1F9A95E1F7ED5CFA4FC181A1
:1036C0008C2F0E945D19CC0FCC0FC0932505209143
:1036D0003F04E22FFF2783E0EE0FFF1F8A95E1F7FB
:1036E000ED5CFA4FC281C093260580916000992756
:1036F00083309105B9F08430910534F4813091051F
:1037000089F00297ECF462C08530910509F45BC042
:10371000853091050CF444C086309105E9F1079796
:1037200011F154C0E22FFF27C3E0EE0FFF1FCA952F
:10373000E1F7ED5CFA4FC2818C2F0E94771946C0E9
:103740008C2F0E947E1980913F04E82FFF27B3E061
:10375000EE0FFF1FBA95E1F7ED5CFA4FC3818C2F96
:103760000E94A11933C08C2F0E947E1980913F04C2
:10377000E82FFF27A3E0EE0FFF1FAA95E1F7ED5C0E
:10378000FA4FC3818FE70E94A1198C2F0E94B419B0
:103790008C2F0E94F0191AC08C2F0E94871A16C015
:1037A0008C2F0E94F31980913F04E82FFF2773E0CC
:1037B000EE0FFF1F7A95E1F7ED5CFA4FC3818C2F76
:1037C0000E94691A03C08C2F0E94F319CF910895AB
:1037D000DF92EF92FF920F931F93CF93DF93F9B293
:1037E00086B3E3B2D0B283E00E94FF1F082F00959A
:1037F000CF2DDD27C4FD05C0802F869586950E94BC
:103800004519C5FD14C0102F16951695812F0E94DD
:10381000451980913F04E82FFF2763E0EE0FFF1F5B
:103820006A95E1F7ED5CFA4F108300932405C6FD1D
:1038300014C08091600099270497202F2695269523
:10384000029740F4822F0E945D19809150060E94D9
:10385000F31903C0822F0E945D19F7FC22C0009368
:10386000250580913F04E82FFF2753E0EE0FFF1F4F
:103870005A95E1F7ED5CFA4F202F26952695218386
:103880008091600099270497029740F4822F0E944C
:103890005D19809150060E94F31903C0822F0E9487
:1038A0005D19CE2DDD27C6FD27C0809160009927C8
:1038B0008630910564F4843091059CF48230910542
:1038C000A1F0833091054CF4019739F015C0863092
:1038D000910579F0079749F00FC0802F0E94771962
:1038E0000BC0802F0E94F31907C0802F0E947E1901
:1038F00003C0802F0E94871AC5FD35C0009326059E
:1039000080913F04E82FFF2743E0EE0FFF1F4A9509
:10391000E1F7ED5CFA4F02838091600099278630D1
:10392000910564F4843091059CF482309105A1F0F6
:10393000833091054CF4019739F015C0863091051C
:1039400079F0079749F00FC0802F0E9477190BC0BC
:10395000802F0E94F31907C0802F0E947E1903C098
:10396000802F0E94871AC2FD26C08091600099278F
:103970008330910501F18430910534F48130910553
:10398000D1F0029739F017C08430910589F007977C
:1039900029F011C0802F0E94A1190DC08FE70E944D
:1039A000A119802F0E94B419802F0E94F01903C022
:1039B000802F0E94691AC3FD32C080913F04E82F16
:1039C000FF2733E0EE0FFF1F3A95E1F7ED5CFA4F6A
:1039D00003838091600099278330910501F1843041
:1039E000910534F481309105D1F0029739F017C078
:1039F0008430910589F0079729F011C0802F0E942B
:103A0000A1190DC08FE70E94A119802F0E94B4193F
:103A1000802F0E94F01903C0802F0E94691AD7FCE2
:103A200009C0802F8F738093360402950695077026
:103A300000936000DF91CF911F910F91FF90EF9065
:103A4000DF90089580913B0690913C0601969093FB
:103A50003C0680933B06089578941F920F920FB610
:103A60000F921124EF92FF920F931F932F933F9386
:103A70004F935F936F937F938F939F93AF93BF9376
:103A8000CF93EF93FF93F89480913D068F5F8093DF
:103A90003D0686B399278470907095958795959586
:103AA0008795282F80913B0690913C06449710F013
:103AB000213031F4809140048F5F809340041DC118
:103AC000959A80917006880F880F880F887180936F
:103AD0003F040E94401BC0917006CF5FC0937006E8
:103AE00080E390E090937D0080937C00C13099F456
:103AF00010923E0610923F06109240061092410628
:103B0000109252061092600610925F0610923C06C8
:103B100010923B06F1C024B52093520680913B06DB
:103B200090913C069093600680935F06AA27BB277E
:103B300080935A0690935B06A0935C06B0935D0653
:103B4000E22EFF2400271127E0921105F0921205C2
:103B5000009313051093140520917800309179009B
:103B600040917A0050917B00BC01CD010E94B421AC
:103B70009B01AC0160932C0570932D0580932E055D
:103B800090932F0580913E0690913F06A0914006AC
:103B9000B09141068093630690936406A0936506F6
:103BA000B0936606E0923706F09238060093390625
:103BB00010933A06280F391F4A1F5B1F2E0D3F1D19
:103BC000401F511F20933E0630933F06409340060E
:103BD0005093410610923C0610923B0614BC8C2F69
:103BE000992701977C010027F7FC0095102FE092A0
:103BF0002705F09228050093290510932A05CA018C
:103C0000B901A80197010E94E72179018A01E3E047
:103C1000EE0CFF1C001F111FEA95D1F7E09218056A
:103C2000F092190500931A0510931B052FEF3FEF33
:103C300040E050E020932005309321054093220579
:103C400050932305C801B7010E94E7212F5F3F4F22
:103C50004F4F5F4F20938206309383064093840634
:103C600050938506C801B7010E94E72120934806BA
:103C70003093490640934A0650934B068091720058
:103C800090917300892F99278BBD809172008ABD16
:103C90006091820670918306709375006093740042
:103CA000809148069091490690937300809372002A
:103CB000689F9001699F300D789F300D1124C901D4
:103CC0009C0144275527D801C701821B930BA40BE5
:103CD000B50B8093760690937706A0937806B09301
:103CE0007906CB01AA27BB2780934306909344060D
:103CF000A0934506B09346069598FF91EF91CF911A
:103D0000BF91AF919F918F917F916F915F914F91F3
:103D10003F912F911F910F91FF90EF900F900FBE49
:103D20000F901F9018958F929F92AF92BF92CF9253
:103D3000DF92EF92FF920F931F93CF9381E00E9447
:103D40004E0FDC01CB01181619060CF04CC14C01CA
:103D5000E0904306F0904406009145061091460617
:103D60000894E11CF11C011D111DE0924306F09224
:103D700044060093450610934606A0901805B0909F
:103D80001905C0901A05D0901B05C601B501A80100
:103D900097010E94E72120936706309368064093BD
:103DA000690650936A06CA01B901A80197010E94E9
:103DB000B421DC01CB01A81AB90ACA0ADB0AA09215
:103DC0007106B0927206C0927306D09274068DE8A6
:103DD00098E09F938F93C1E0CF930E94F1070F90DB
:103DE0000F900F9084EA98E09F938F93CF930E9457
:103DF000F1078091760690917706A0917806B091B0
:103E00007906BC01CD010E94C8160F900F900F904B
:103E100089EB98E09F938F93CF930E94F1070F90C7
:103E20000F900F908CEB98E09F938F93CF930E940D
:103E3000F1078091180590911905A0911A05B0918C
:103E40001B05BC01CD010E94C8160F900F900F906A
:103E500081ED98E09F938F93CF930E94F1070F908D
:103E60000F900F9084ED98E09F938F93CF930E94D3
:103E7000F1078091430690914406A0914506B091C8
:103E80004606BC01CD010E94C8160F900F900F90FE
:103E900089EE98E09F938F93CF930E94F1070F9044
:103EA0000F900F908CEE98E09F938F93CF930E948A
:103EB000F1078091670690916806A0916906B0911C
:103EC0006A06BC01CD010E94C8160F900F900F909A
:103ED00081E099E09F938F93CF930E94F1070F9019
:103EE0000F900F9084E099E09F938F93CF930E945F
:103EF000F1078091710690917206A0917306B091BE
:103F00007406BC01CD010E94C8160F900F900F904F
:103F100089E199E09F938F93CF930E94F10780915D
:103F2000710690917206A0917306B0917406BF77E6
:103F30008093710690937206A0937306B0937406F3
:103F40000F900F900F908CE199E09F938F93CF93F8
:103F50000E94F1078091710690917206A0917306FC
:103F6000B0917406BC01CD010E94C8160F900F904D
:103F70000F9081E399E09F938F93CF930E94F10775
:103F8000209171063091720640917306509174062B
:103F90008091760690917706A0917806B091790687
:103FA0000F900F900F90281739074A075B0750F4BE
:103FB00084E399E09F938F93CF930E94F1070F9032
:103FC0000F900F9082E499E09F938F93CF930E947C
:103FD000F1070F900F900F900894810891088114B9
:103FE000910409F0B5CECF911F910F91FF90EF9002
:103FF000DF90CF90BF90AF909F908F9008950F93D8
:104000001F93CF93DF93082FC0E0D0E010E0802F04
:104010000E942C0CC80FD91F1F5F1830C0F3A5E0F9
:10402000D695C795AA95E1F78C2F9927DF91CF9167
:104030001F910F910895809130058F5F8093300517
:1040400090912405981710F4C29801C0C29A9091DB
:10405000300580912505891710F4C09801C0C09AD9
:1040600080912605891710F4C1980895C19A089582
:10407000089581E00E944E0FDC01CB01809324055E
:1040800082E00E944E0FDC01CB018093250583E086
:104090000E944E0FDC01CB01809326050895FB01A1
:1040A000DC0101900D920020E1F70895FB01DC0195
:1040B0004150504030F08D910190801919F400204A
:1040C000B9F7881B990B08952F923F924F925F92F8
:1040D0006F927F929F92AF92BF92CF92DF92EF92B8
:1040E000FF920F931F93CF93DF93CDB7DEB76E97F9
:1040F0000FB6F894DEBF0FBECDBF898B9A8B6B8B4A
:104100007C8B4D8B5E8B3C011F8A188EF301919046
:104110003F01892D99270E943A22892BB9F70DE298
:10412000901609F4FFC01BE2911609F4F7C02D891F
:104130003E892115310509F4DAC02031310509F431
:10414000D6C0ED89FE89EF2B41F430E3931609F4D4
:10415000C9C04AE050E04D8B5E8B8D899E89AA27AD
:1041600097FDA095BA2F898F9A8FAB8FBC8F8F89BF
:10417000988D892B09F4B1C060E070E080E090E890
:10418000298D3A8D4B8D5C8D0E94092229873A87B3
:104190004B875C876D877E878F87988B58E0DE0121
:1041A0001196FE01399601900D925A95E1F7CC24B3
:1041B000DD247601AA24BB2429803A804B805C80D0
:1041C0002D813E812D8F3E8F092D1127C8010E9420
:1041D0002E22892BC9F1C8010E943322892B09F4B0
:1041E0006BC070ED970E892D99276D897E89861792
:1041F000970754F5B7FC24C02C143D044E045F040B
:10420000F8F0C214D304E404F504A9F021E0A22ECE
:10421000B12CC701B601298D3A8D4B8D5C8D0E9462
:10422000B4216B017C01C90CD11CE11CF11CD30130
:104230009D903D01C9CFAD8CBE8CA816B90634F750
:104240003FEFA32EB32EF3CFB7FE29C0EF89F88D31
:10425000EF2BE1F0C12CD12CE12C90E8F92E02E2F9
:1042600010E010938706009386068B899C89892B22
:1042700009F460C0AB2839F0C3010197AB89BC8950
:104280008D939C9357C089899A89F8CF8FEFC82E58
:104290008FEFD82E8FEFE82E8FE7F82EE0CFAF8983
:1042A000B88DAB2B11F3F094E094D094C094C11C62
:1042B000D11CE11CF11CD9CFC8010E942622892BF8
:1042C00019F2C8010E942422892B21F0802F8753E4
:1042D000982E89CF802F8755FBCF6FEF7FEF8FEF21
:1042E0009FE74ECF08E010E00D8B1E8B36CF40E3EA
:1042F000941609F026CFF3018081883719F08835AC
:1043000009F01FCFD30111969C9082E090E0680ED7
:10431000791E60E170E06D8B7E8B13CFD3019D9091
:104320003D0105CF21E030E02F8B388FF3019190D4
:104330003F01FDCEC701B6016E960FB6F894DEBF01
:104340000FBECDBFDF91CF911F910F91FF90EF90E6
:10435000DF90CF90BF90AF909F907F906F905F90D5
:104360004F903F902F900895629FD001739FF0016E
:10437000829FE00DF11D649FE00DF11D929FF00DF5
:10438000839FF00D749FF00D659FF00D9927729F2C
:10439000B00DE11DF91F639FB00DE11DF91FBD01B7
:1043A000CF0111240895AA1BBB1B51E107C0AA1F0E
:1043B000BB1FA617B70710F0A61BB70B881F991FC6
:1043C0005A95A9F780959095BC01CD010895A1E279
:1043D0001A2EAA1BBB1BFD010DC0AA1FBB1FEE1F7F
:1043E000FF1FA217B307E407F50720F0A21BB30BCA
:1043F000E40BF50B661F771F881F991F1A9469F746
:1044000060957095809590959B01AC01BD01CF01A1
:10441000089597FB092E05260ED057FD04D0D7DF4F
:104420000AD0001C38F450954095309521953F4FA7
:104430004F4F5F4F0895F6F7909580957095619571
:104440007F4F8F4F9F4F089585FD23C08062992332
:1044500001F58136F4F08B37E4F408959923C9F41B
:104460008095807808959923A1F4803394F08A335D
:1044700084F40895992369F4803269F08A3059F000
:104480008C3049F08D3039F0893029F08B3009F4C7
:0A4490000895992788270895FFCFAB
:10449A0002010001000A00E803036300350011006D
:1044AA000100EBFB0E00FF00FF0000000A00686538
:1044BA006C700064756D7061726773310064756D3C
:1044CA007061726773320064756D706172677333FD
:1044DA0000617265660061766363007061007062F4
:1044EA000070630070640061646300707000646748
:1044FA000067007373007369007469636B73006902
:10450A006D7000776176007065720064697600727A
:10451A007065720066696C006678006F64006C648E
:08452A000065786572000100D4
:00000001FF
